:10000000D8C0002055070000530700005307000028
:1000100053070000530700005307000000000000D2
:100020000000000000000000000000005307000076
:1000300053070000000000005307000053070000B2
:100040005307000053070000530700005307000048
:100050005307000053070000530700005307000038
:1000600053070000530700005307000095080000E5
:100070005307000053070000530700005307000018
:100080005307000053070000530700005307000008
:1000900053070000530700005307000053070000F8
:1000A00053070000530700005307000053070000E8
:1000B00053070000530700005307000053070000D8
:1000C00053070000530700005307000053070000C8
:1000D00053070000530700005307000053070000B8
:1000E000530700005307000000000000000000005C
:1000F000000000001907000053070000530700002C
:100100005307000053070000530700005307000087
:100110005307000053070000530700005307000077
:100120005307000053070000530700005307000067
:100130005307000053070000530700005307000057
:100140005307000053070000530700005307000047
:100150005307000053070000530700005307000037
:100160005307000053070000530700005307000027
:100170005307000053070000530700005307000017
:100180005307000053070000530700005307000007
:1001900053070000530700005307000053070000F7
:1001A00053070000530700005307000053070000E7
:1001B00053070000530700005307000053070000D7
:1001C00053070000530700005307000053070000C7
:1001D00053070000530700005307000053070000B7
:1001E00053070000530700005307000053070000A7
:1001F0005307000053070000530700005307000097
:100200005307000053070000530700005307000086
:100210005307000053070000530700005307000076
:100220005307000053070000530700005307000066
:100230005307000053070000530700005307000056
:100240005307000053070000530700005307000046
:100250005307000053070000530700005307000036
:100260005307000010B5054C237833B9044B13B184
:100270000448AFF300800123237010BD0800002064
:1002800000000000FC10000008B5034B1BB103493F
:100290000348AFF3008008BD000000000C00002000
:1002A000FC10000038B5044600380C4B0D4618BF52
:1002B00001200B494FF4E07298472368AB4208D005
:1002C0004BB9084B25602046984740F2B273A361B2
:1002D00038BD0020FCE76FF01100F9E7B904000019
:1002E000DC0F000019080000024A0348034B111DEF
:1002F000184700BF00000020C000002001030000DC
:1003000010B5044B04249C76FF241C71C3E9020140
:100310005A6310BD2400002038B50D46044610B1C4
:10032000081E18BF01200A490A4B4122984720465F
:10033000094B40F8045F29469847002807DB4FF433
:100340000043A382054B2361054BE360002038BDC9
:10035000F60F0000B9040000550D0000D90300009D
:10036000A103000030B50C4685B0054610B1081E4B
:1003700018BF0120B4220749074B9847236801930F
:1003800063680293A368039301A9044B281D98474F
:1003900005B030BDF60F0000B9040000890E000062
:1003A0007FB50446003818BF01200E4615460749A0
:1003B000074BA42298470023CDE9016301A9054B0F
:1003C0000395A4F10C00984704B070BDF60F00002F
:1003D000B9040000650300007FB50446003818BF6B
:1003E00001200E4615460749074B882298470023EF
:1003F000019301A9054B0296A4F10C0003959847BF
:1004000004B070BDF60F0000B904000065030000E1
:1004100070B50D46044610B1081E18BF01200549ED
:10042000054B3122984729462046044BBDE87040D1
:10043000184700BF12100000B90400009905000021
:10044000094A138810B59BB21380084B9847084B94
:100450009847084B9847084B9847BDE81040074B12
:1004600040F6FF70184700BF00400041F107000050
:10047000C10400000D070000D90400008104000041
:10048000C20707D5094B0A4A1A6243F6FD7259683A
:100490001142FCD1030707D5044B064ADA6243F642
:1004A000FD7259681142FCD1704700BF001C00402A
:1004B000010101000501010000B900BE7047000004
:1004C000034B044A9A611A699207FCD5704700BF32
:1004D00000100040062600032C4A136A23F00F0385
:1004E00043F00403136243F6FD7351681942FCD1D3
:1004F00053685807C3F38001FAD4254B254A19776E
:100500009A6293F82C20C2F30011D206F9D483F832
:1005100020101F4B93F82C205007FBD402221A778F
:100520001B4B93F82C209107FBD45A6A5A62184B44
:1005300093F82C201207FBD49F2283F82020144B21
:1005400093F82C205007FBD493F82020D10719D51D
:100550001A6902F41062B2F5106FF9D10B4A5368B0
:10056000002BFCD1136A23F00F0343F00103136245
:1005700043F6FD7351681942FCD1044A53685B0786
:10058000FCD470471A69D205FCD5E7E7001C00408F
:10059000001000400000010438B50C46054610B1BB
:1005A000081E18BF0120124B1249D822984794F810
:1005B0002F302C6043F0010384F82F3094F82F0083
:1005C00010F00100FAD10E2384F82E300F2384F8A6
:1005D0002930A38E9BB26FEA53236FEA4323A3868D
:1005E000E38E9BB26FEA93236FEA8323E38638BDE1
:1005F000B90400002C1000002DE9F8430E46154602
:10060000044618B129B3101E18BF01201249134B1C
:10061000134FF12298470834B9462046B8470028BE
:10062000FBD0DFF844800027F15D2046C04720461C
:10063000C8470028FBD00137BD42F5D8002D094E30
:1006400008BF01252046B0470028FBD02846BDE85A
:10065000F8830846DAE700BF43100000B904000041
:10066000370D0000410D0000290D00002DE9F84371
:100670000E461546044618B1E9B1101E18BF0120F8
:100680000E490F4BDFF83C90DFF83C804FF4867248
:100690009847002708342046C8470028FBD020464A
:1006A000C047F0550137BD42F5D8002D14BF28468C
:1006B0000120BDE8F8830846E2E700BF43100000D0
:1006C000B90400004B0D00002F0D000038B50D4699
:1006D000044610B1081E18BF01200749074B3422F9
:1006E0009847074B294604F10800984718B9054B6D
:1006F0006360054B236038BD43100000B90400005F
:10070000FD0C00006D060000F9050000014B012200
:100710005A717047000800400B4A937882B0DBB2F0
:100720000193019B990705D5084B1B6813B15068CD
:1007300002B01847019BDB0704D5044B5B680BB183
:10074000014AF4E702B07047000002416000002057
:100750007047FEE718491948814210B50AD0184B76
:10076000DA1C121A22F00302C41EA34238BF002270
:10077000144B9847144B1548DA1C121AC11E22F06C
:100780000302994288BF0022114B00219847114A69
:10079000114B22F07F029A60D3F8882042F4700255
:1007A000C3F88820BFF34F8FBFF36F8F0B4B984771
:1007B0000B4B9847FEE700BFFC1000000000002034
:1007C00008000020B10F0000D80000200800002021
:1007D000CD0F00000000000000ED00E0690F0000F8
:1007E000E507000008B5014B9847FEE7490F0000F8
:1007F000064B42F286029A8200229A75DA75DA690D
:1008000002F47C52DA6101221A747047001400402D
:1008100003690B42FCD1704710B5044618B100685B
:10082000003818BF01201749174B2F229847174B44
:100830002068174A1C6048F20301904703889B0711
:100840000AD52068038823F002031B041B0C0380D5
:100850009047206802219047206803889BB243F0AC
:1008600001030380012190472068904720684FF4DE
:100870000143038048F20301904723680020186673
:1008800010BD00BF5F100000B90400007000002020
:10089000110800000D4B10B51C682268918953891E
:1008A0009BB20B40DA0507D563682046984723685A
:1008B0004FF480729A8110BD5B04FCD5A36820467A
:1008C000984723684FF48042F4E700BF700000208F
:1008D00000F01F0330B501259D4040090D4BC001BC
:1008E0000229ACB24FEA154203440BD044F08044D5
:1008F00044F4003442F040425D6042F400329C62B5
:100900009A6230BD44F080449D6042F040429C6257
:10091000F6E700BF00800041420900F01F0303EB2F
:10092000C21303F1824303F5004393F8402002F021
:10093000FB0283F8402070474309DB0103F1824347
:1009400030B503F5004300F01F041D1903EB5403F9
:1009500095F8402002F0FE0242F0010285F84020A6
:10096000CAB293F8301010F0010F1BBF01F00F0155
:1009700041EA021101F0F001C9B208BF114383F846
:10098000301030BD024A536943F40073536170471D
:100990000008004010B5044B044905489847BDE8DD
:1009A0001040044B184700BF850900000024004098
:1009B00078000020A502000010B5054C0549042070
:1009C000A04723460449BDE810400520184700BF52
:1009D000390900000300040003000500064B402213
:1009E000C3F89C204322C3F88C20044A536943F483
:1009F00080535361704700BF001C00400008004056
:100A000010B5054B054906489847064B0022984704
:100A1000BDE81040044B1847DD09000000300040DD
:100A200098000020CD060000B909000070B5124EF4
:100A3000124D134C4FF48033C6F81431022150206C
:100A4000A84701F5A0015020A0474FF40033C6F895
:100A5000143102215120A84701F5A2015120A047DD
:100A600001215220A847074B0749522098472346A7
:100A7000BDE87040184700BF00800041D108000069
:100A8000390900001909000002005200064B4022FB
:100A9000C3F810214322C3F88C20044A136A43F0A0
:100AA00004031362704700BF001C004000080040B0
:100AB00010B5054B054906489847064B9847BDE8D1
:100AC0001040054B184700BF8D0A00000008004386
:100AD000A4000020190300002D0A00002DE9F047B2
:100AE000214E224F224D234C4FF4006902212B202E
:100AF000B8472B202049C6F89490A847A047022168
:100B00000820B8474FF48073736108204FF0081134
:100B1000A847A04702210920B8474FF4007373612A
:100B200009201649A8474FF48068A04702210A20EF
:100B3000B8470A201249C6F81480A847A0470221E6
:100B40000B20B8470B200F49C6F81490A847A047C0
:100B500002212A20B847C6F894802A20A8470A49CB
:100B60002346BDE8F047184700800041D108000047
:100B7000190900003909000008002B0008000900CD
:100B800008000A0008000B0008002A00054A136943
:100B900043F400431361044B4022C3F83421C3F8EB
:100BA0008C20704700080040001C004010B5054B29
:100BB000054898474FF08A41044B9847BDE81040DC
:100BC000034B18478D0B0000C000002011040000EB
:100BD000DD0A000010B5064B9847064B9847064BB8
:100BE0009847064B9847BDE81040054B184700BF93
:100BF0004104000095090000010A0000B10A00004C
:100C0000AD0B0000C3690B42FCD17047C3690B42B6
:100C1000FCD170470268034B22F0020202600321FC
:100C2000184700BF050C00000268034B22F00202C7
:100C300002600321184700BF0D0C000070B50C4D79
:100C400006460FCD88B06C460FC495E80F0084E8C7
:100C50000F006A46002352F8041BB14202D1D8B2F9
:100C600008B070BD0133082BF5D10020F8E700BFB4
:100C70009010000038B51A4B0446984728B119491E
:100C8000194B40F2472200209847E369174D13F0B3
:100C9000010F0ED103212046A84723689B0703D5E7
:100CA000134B98470221A8470523236003212046C0
:100CB000A84720460121A8470E4B23600321A847DF
:100CC0004FF4403363601F21A8470B4BA3604FF6DE
:100CD000B943A3810023A373184684F8303038BD8C
:100CE0003D0C000074100000B90400000D0C000061
:100CF000290C0000040010400200700070B5054689
:100D000000380C46054B064918BF0120BB22984706
:100D10002C602046034BBDE870401847B904000022
:100D200074100000750C0000036899627047036836
:100D3000986AC0B270470368187E00F001007047DF
:100D40000368187EC0F3400070470368187EC0F344
:100D5000800070472DE9F843444B454D074608464F
:100D60000C469847062818BF0025002F5DD0201E8E
:100D700018BF01203F4E404940F63F12B047B046F1
:100D8000002D70D0E3693D4E13F0010F13D1032104
:100D90002046D5F80090B04723689B0709F01C094E
:100DA00003D5374B98470221B04749F00103236030
:100DB00003212046B04701212046B0472B68DFF8C9
:100DC000C4903C6003F01C03082B30D12A49012059
:100DD00040F61D12C0472B6803EA09032360032174
:100DE0002046B0476B6823F4083323F4107343F4B0
:100DF000003343F4107363601721B047AB6863623C
:100E00006B7B84F83030E369002BFCD16B6813F006
:100E1000070F0CBF012302233B71AB7BEA7B43EA44
:100E20000223FB800020BDE8F8833846A2E7124980
:100E3000012040F60912C0472B6803EA090323602A
:100E400003212046B0476B6823F4383323F4107332
:100E500043F4003363601721B0472B7B23736B7B14
:100E600084F83030D2E76FF00C00DCE73D0C000076
:100E7000C8100000B904000074100000050C000048
:100E8000150C0000FCFEFFFF2DE9F843046890F804
:100E900004802A4B0746201ED1E9006540F6A322B4
:100EA00018BF0120894626499847E26912F00702D7
:100EB0003ED1244B032120469847236899073AD511
:100EC0001146237ED8B25B070FD48A4218D8C307D5
:100ED00016D5FB8836B1B8F1010F33788CBF36F8E0
:100EE000023B01360132A3620AE0A36A3DB1B8F1C8
:100EF000010F2B7085BF1B0A6B7001350235013164
:100F0000000607D4D9F808309342DAD88B42D8D8F3
:100F1000104606E04FF6FF736383802323766FF05D
:100F20001200237E9B07FCD003232376BDE8F883C1
:100F30006FF00300FAE76FF01300F7E7B904000061
:100F400074100000050C000010B5044B9847044BCA
:100F50009847BDE81040034B184700BFD50B000071
:100F6000E90200005107000070B50D4D0D4C641BE7
:100F7000A4100026A64209D10B4D0C4C00F0AEF88F
:100F8000641BA4100026A64205D170BD55F8043B91
:100F900098470136EEE755F8043B98470136F2E7EB
:100FA000E8100000E8100000E8100000EC1000005D
:100FB0000A44914200F1FF3300D1704710B511F897
:100FC000014B03F8014F9142F9D110BD0244034691
:100FD000934200D1704703F8011BF9E72E2E2F68CA
:100FE000616C2F7372632F68616C5F63616C656EF7
:100FF0006461722E63002E2E2F68616C2F737263F2
:101000002F68616C5F7370695F6D5F73796E632EBB
:1010100063002E2E2F68616C2F7372632F68616CD2
:101020005F6D63695F73796E632E63002E2E2F6888
:10103000706C2F736468632F68706C5F736468638F
:101040002E63002E2E2F68616C2F7372632F6861E0
:101050006C5F75736172745F73796E632E63002EBB
:101060002E2F68706C2F7274632F68706C5F7274AF
:10107000632E63002E2E2F68706C2F736572636F62
:101080006D2F68706C5F736572636F6D2E63000007
:101090000030004000340040002001410040014188
:1010A000000000430004004300080043000C00431C
:1010B0000000000000000000000000000000000030
:1010C00000000000000000000C00200000000200F2
:1010D00000000000FE00FF0106000000F8B500BFA0
:1010E000F8BC08BC9E46704789020000F8B500BFF6
:0C10F000F8BC08BC9E467047650200007A
:0810FC00FFFF0100FFFF0000EF
:00000001FF
